:100000000C941E060C949E280C94CB280C94460647
:100010000C9446060C9446060C9446060C94460630
:100020000C9446060C9446060C941B130C9446063E
:100030000C9446060C9446060C9446060C94460610
:100040000C94F8280C9446060C94E62C0C94292D5C
:100050000C9446060C9446060C9446060C944606F0
:100060000C9446060C944606FD185F193E1941197A
:10007000441947194A194D1950195F195919911AFC
:10008000931A931A911A931A931A931A931A931A0A
:10009000931A931A931A931A931A931A931A931AF8
:1000A000171A931A931A931A931A931A8819931A70
:1000B000931A931A931A931A931A931A931A931AD8
:1000C000931A931A931A931A931A931A231A231AA8
:1000D000231A231A231A231A231A231A231A931AC8
:1000E000931A931A931A931A931A8819221A221A96
:1000F000221A221A931A301A361A3C1A421A481A2D
:100100004E1A541A5A1A641A6E1A781A821AC9198F
:100110008B19931A931A931A931A171A931A931AFC
:10012000931A931A931A931A931A931A211A211A4B
:10013000211A211A931A301A361A3C1A421A481AEE
:100140004E1A541A5A1A641A6E1A781A821AC9194F
:100150008B19931A931A931A931A171AC61AC61A56
:10016000C61AC61AC61AC61AC61AC61AC61AC61A8F
:10017000C61AC61AC61ADD1BDD1BDD1BDD1BDD1B07
:10018000DD1B0B1B151B1F1B291B871B911BA01B9A
:10019000B11B391D4E1D5A1D631D721D971DA01DDB
:1001A000E91DB21DFB20012107210E211C213E214A
:1001B0005C21456E746572206D656E752E2E2E0065
:1001C000546F67676C6564206D6963726F50504D42
:1001D00000546F67676C656420696E76657274653C
:1001E000642050504D2100546F67676C6564205443
:1001F00058206D7574696E672100546F67676C6570
:10020000642074656C656D65747279210050726F3D
:10021000746F636F6C206572726F72207769746897
:100220002052580054696D656F7574207768656E4B
:1002300020636F6E6E656374696E6720746F205201
:100240005800507265737320616E79206B65792058
:10025000746F2063616E63656C00436F6E6E6563DF
:1002600074696E6720746F2052582C20706F776508
:100270007220757020746865205258202877697440
:10028000682062696E6420706C7567206966206EF4
:100290006F74207573696E6720616C776179732064
:1002A00062696E642900546F67676C656420276912
:1002B0006D6D656469617465206F75747075742700
:1002C00000546F67676C65642027736C61766520E6
:1002D0006D6F64652700546F67676C6564202761E4
:1002E0006C776179732062696E642700546F676769
:1002F0006C65642050504D206368616E6E656C20A3
:100300006C696D69740053657420525353492069B8
:100310006E6A656374696F6E206368616E6E656C8A
:100320002028303D3D64697361626C652900536526
:10033000742050504D206D696E696D756D20737914
:100340006E630053657420626561636F6E20696E31
:1003500074657276616C0053657420626561636FC9
:100360006E2064656C617900536574206265616319
:100370006F6E206672657175656E637920696E2097
:10038000487A3A20303D64697361626C652C205074
:10039000783D504D52206368616E6E656C20782CFC
:1003A0002046783D465253206368616E6E656C202E
:1003B00078005365742050574D2073746F7020641B
:1003C000656C61792028302064697361626C6564B2
:1003D0002C20312D323535203D3D20302E317320FB
:1003E0002D2035306D696E29005365742050504DB5
:1003F0002073746F702064656C61792028302064EC
:10040000697361626C65642C20312D323535203D75
:100410003D20302E3173202D2035306D696E29003E
:10042000536574206661696C736166652064656CF0
:1004300061792028302064697361626C65642C20C6
:10044000312D323535203D3D20302E3173202D2089
:1004500035306D696E29002A2A2A2A2A2A2A2A2A50
:100460002A2A2A2A2A2A2A2A2A2A2A2A2A2A2A2AEC
:100470002A2A2A2A0052582041636B6564202D20C5
:1004800072657665727420737563636573736675E0
:100490006C21002A2A2A2A2A2A2A2A2A2A2A2A2AAD
:1004A0002A2A2A2A2A2A2A2A2A2A2A2A2A2A2A2AAC
:1004B000002A2A2A2A2A2A2A2A2A2A2A2A2A2A2AC6
:1004C0002A2A2A2A2A2A2A2A2A2A2A2A2A2A00528E
:1004D000582041636B6564202D20757064617465DC
:1004E000207375636365737366756C21002A2A2A0D
:1004F0002A2A2A2A2A2A2A2A2A2A2A2A2A2A2A2A5C
:100500002A2A2A2A2A2A2A2A2A2A0056616C696457
:100510002063686F69636573206172653A205B319F
:100520005D2D5B31365D20286368616E6E656C20E1
:10053000312D31362900536574206F7574707574D0
:1005400020666F7220706F727420005B585D2061AE
:10055000626F7274206368616E67657320616E6498
:10056000206578697420525820636F6E6669670051
:100570005B535D20736176652073657474696E6783
:100580007320746F205258005B525D20726576654F
:1005900072742052582073657474696E6773207486
:1005A0006F2064656661756C747300557365206EA9
:1005B000756D62657273205B312D445D20746F2010
:1005C0006564697420706F727473205B452D515D92
:1005D00020666F722073657474696E677300202DD6
:1005E00020726563656976657220636F6E66696700
:1005F000757261746F722C20727820737720000AF4
:100600000A6F70656E4C52536E67200053657420FC
:1006100073657269616C2062617564726174653AB8
:10062000200056616C69642063686F696365733A82
:100630002031202D20342B34202F2032202D203823
:10064000202F2033202D20382B34202F2034202D14
:10065000203132202F2035202D2031322B34202FF5
:100660002036202D20313600536574204368616E9A
:100670006E656C20636F6E6669673A20005365741F
:100680002044617461726174652028302D32293AEA
:10069000200053657420486F70206368616E6E653A
:1006A0006C7320286D61782032342C207365706162
:1006B000726174656420627920636F6D6D61732966
:1006C0002076616C69642076616C75657320312DCC
:1006D0003235353A2000536574206368616E6E656B
:1006E0006C2073706163696E6720287831306B48C5
:1006F0007A293A200053657420524620706F77653E
:10070000722028302D37293A200053657420524634
:10071000206D6167696320286865782920652E67E8
:100720002E20307844454144463030443A2000532E
:1007300065742062617365206672657175656E63AC
:10074000792028696E20487A293A20005B5A5D207A
:10075000656E746572207265636569766572206383
:100760006F6E66696775726174696F6E2075746902
:100770006C79005B465D20646973706C61792061FF
:10078000637475616C206672657175656E63696509
:10079000732075736564005B525D2063616C6375E3
:1007A0006C6174652072616E646F6D206B65792079
:1007B000616E6420686F70206C697374005B495DC2
:1007C000207265696E697469616C697A6520736508
:1007D0007474696E677320746F20736B65746368DB
:1007E0002064656661756C7473005B585D2072658A
:1007F00076657274206368616E67657320616E64EC
:100800002065786974206D656E75005B535D20739B
:100810006176652073657474696E677320746F20E8
:10082000454550524F4D20616E64206578697420B3
:100830006D656E7500557365206E756D62657273BA
:10084000205B302D395D20746F20656469742070E1
:100850006172616D657465727300202D2053797328
:1008600074656D20636F6E66696775726174696F18
:100870006E000A0A6F70656E4C52536E672000510D
:1008800029204F7574707574206265666F726520DB
:100890006C696E6B20283D465329203A2000502970
:1008A00020536C617665206D6F64652028657870D3
:1008B0006572696D656E74616C293A20004F29205C
:1008C00054696D65642042494E44206174207374FC
:1008D000617274757020203A20004E292050504DCE
:1008E000206F7574707574206C696D69746564200F
:1008F000202020203A200044495341424C454400E6
:100900004D292050504D205253534920746F20637D
:1009100068616E6E656C202020203A20004C2920F2
:1009200050504D206D696E696D756D2073796E63E1
:10093000202875732920203A200044495341424C15
:100940004544004B29204661696C736166652062ED
:100950006561636F6E20696E74762E2028312D32AA
:10096000353573293A20004A29204661696C736144
:10097000666520626561636F6E2064656C617920D5
:1009800028302D323535203D3E20313073202D204A
:100990003135306D696E293A200049292046616958
:1009A0006C7361666520626561636F6E206672714B
:1009B0002E203A200048292050574D2073746F7024
:1009C0002064656C6179202020202020203A2000BE
:1009D00047292050504D2073746F702064656C61FE
:1009E00079202020202020203A200046292046611E
:1009F000696C736166652064656C617920202020D4
:100A00002020203A200050574D206368616E6E65AB
:100A10006C200066756E6374696F6E3A2000292041
:100A2000706F72742000506F776572546F776572C3
:100A300000445446205548462033322D62697420C4
:100A400031306368004F70656E4C52536E67525878
:100A5000206D696E6920342F36636800466C7974A6
:100A6000726F6E2F4F72616E6765525820554846FF
:100A70002038636800525820747970653A20004429
:100A8000697361626C656400487A00203D3D200016
:100A900043616C63756C61746564207061636B6540
:100AA0007420696E74657276616C3A200042292068
:100AB0004D6963726F202868616C66292050504D23
:100AC000202020203A00412920496E766572746505
:100AD000642050504D20696E20202020203A0030A4
:100AE00029204D7574652062757A7A657220286DAB
:100AF0006F73746C79293A003929205365726961E2
:100B00006C2062617564726174653A00736D617224
:100B100074506F7274004672536B79005472616E38
:100B200073706172656E740044697361626C6564B0
:100B30000038292054656C656D657472793A2020FF
:100B40002020202020003729204368616E6E656CCC
:100B500020636F6E6669673A202000362920446161
:100B60007461726174652028302D32293A2020206A
:100B700000352920486F70206368616E6E656C7364
:100B80003A2020202020003429204368616E6E65C1
:100B90006C2073706163696E673A202000332920EE
:100BA000524620706F7765722028302D37293A2001
:100BB0002020003229205246206D616769633A2067
:100BC0002020202020202020003129204261736530
:100BD000206672657175656E63793A202020000089
:100BE00000000700020100000304060000000000EE
:100BF00000000001020408102040800102040810D7
:100C00002001020408102004040404040404040263
:100C10000202020202030303030303000000002395
:100C2000002600290000000000250028002B0000FD
:100C3000000000240027002A0000172E11241FBEE8
:100C4000CFEFD8E0DEBFCDBF13E0A0E0B1E0ECE332
:100C5000F2E602C005900D92A83CB107D9F716E064
:100C6000A8ECB3E001C01D92AE38B107E1F71CE07B
:100C7000CCE3DCE004C02297FE010E94202FCA339F
:100C8000D107C9F70E94532E0C941C310C9400001C
:100C900080917305813019F482E08093730580910F
:100CA0007305833019F484E0809373050895A89543
:100CB0000895DC01ED91FC910190F081E02D099502
:100CC00008952091740530917505382748E0C901D1
:100CD000880F991F37FF06C09C0151E2252750E17C
:100CE000352701C09C01415091F730937505209341
:100CF0007405089588E38093760580E092ECA1E086
:100D0000B0E08093770590937805A0937905B09330
:100D10007A0587E08093830580EC92E9ADEEB9E136
:100D200080937B0590937C05A0937D05B0937E0511
:100D300085E0809384058DEE9EEFADEABEED809355
:100D40007F0590938005A0938105B0938205E5E827
:100D5000F5E080E090E0863028F4DC01AE54BC4F32
:100D60002C9101C020E0219301968831910599F7DB
:100D700082E080939D058AE080939E05089580EC33
:100D800091EDA8E9BBE18093BB059093BC05A093CE
:100D9000BD05B093BE0580E090E0A0E0B0E5809393
:100DA000BF059093C005A093C105B093C205E3ECC5
:100DB000F5E080E081938F5F8031E1F70895A0E056
:100DC000B0E0E5EEF6E00C94E92ED82F0E944E2913
:100DD0006115710581059105C9F30E948C2F109250
:100DE0007F05109280051092810510928205C4E063
:100DF000812C912C54018A94C0907F05D09080055D
:100E0000E0908105F0908205FE2CED2CDC2CCC24AA
:100E10000E94872FA50194010E94C82E6C0D7D1D94
:100E20008E1D9F1D60937F057093800580938105C3
:100E300090938205C15001F7DD2309F450C005E805
:100E400015E0E801A12CB12C62E3C62ED12CE12CD7
:100E5000F12C8881882309F442C0B39419F40E94CC
:100E60007A063DC00E94872FA70196010E94C82ED6
:100E7000E1E0E60FA5E8B5E08A2F801B8A1520F493
:100E80008D918E13F9CFE9CF2091840530E0A0E158
:100E9000B7E20E94602E9B01AC01AE2FB0E00E9431
:100EA0006F2E40907B0550907C0560907D05709082
:100EB0007E05640D751D861D971D4090BB055090E5
:100EC000BC056090BD057090BE05461657066806C5
:100ED000790618F2E993A39488E1A812BACFCDB7A6
:100EE000DEB7E0E10C94052F8436910520F4BC01B7
:100EF00080E090E017C09C018E3B910528F42A55B4
:100F00003109AAE0B0E00CC0823D910528F4245BD1
:100F10003109A4E6B0E004C02D5C3109A8E5B2E0D7
:100F20000E94602EA4E6B0E09B01AC010E946F2EEF
:100F3000089590E08C599F4F0E947407089582E0B5
:100F40008093B00085E08093B10061E083E00E946F
:100F5000FB2960E083E00E94342A08950097C9F0DD
:100F60009C0140E050E068E478EE81E090E00E946F
:100F7000C82E2F3F31054105510529F020F02FEFF4
:100F800030E040E050E02093B3008091B0008061F9
:100F900003C08091B0008F7E8093B000089560E020
:100FA0008CE00E94FB2961E08BE00E94FB2961E05C
:100FB0008DE00E94FB2960E082E00E94FB2961E055
:100FC00084E00E94FB29089542E050E068E476E066
:100FD00080E00E947E280895E3E0F0E089E08093BD
:100FE0005700E491E67081E0E63009F080E0089572
:100FF000CF93DF93C82F0E94EC07882381F0DFB7DF
:1010000081E080937205F8940E94570688E18093EE
:101010006000C0936000C1110E945706DFBFDF91DE
:10102000CF9108958F929F92AF92BF92CF92DF920D
:10103000EF92FF92CF93FC01C0A5EC2FE770F0E098
:10104000E658FC4FA081B0E0C7FF03C024E130E0C8
:1010500002C02FE030E0FC0197A183E1989FF001EE
:101060001124E25CFE4F80809180A280B380A20FA9
:10107000B31F20E43FE14DE750E00E947A2EA50126
:1010800094010E94A62E8C2F887149F469017A017F
:10109000E0EDCE0EE7E0DE1EE11CF11C1BC0C7FF39
:1010A00005C060E47AE88CE29EE004C060E07EEE79
:1010B0008AEB9BE069017A01F8EBCF0EFBE0DF1EC3
:1010C000E11CF11CA50194010E94A62EC20ED31EA4
:1010D000E41EF51EC701B60169517C4F8F4F9F4F2B
:1010E00028EE33E040E050E00E94A62EA8EEB3E0E8
:1010F0000E946F2ECF91FF90EF90DF90CF90BF9026
:10110000AF909F908F9008958F3F910551F048F0D8
:10111000811522E0920738F08115934030F482E087
:10112000089580E0089581E0089583E00895A0E0A7
:10113000B0E0EDE9F8E00C94F22EEB018A01B82F53
:10114000B695A0E028813981F80120832A813B816E
:1011500021832C813D8122832E813F8123836881DD
:1011600079814A815B812C813D81EE81FF819F2FB6
:101170009295990F990F907C272F2370922B252FF2
:101180002370220F220F922B232F23702295207F72
:10119000922BF80194830B5F1F4F2896AF5FBA170D
:1011A00088F680FF24C0888199810E948408D82E07
:1011B0008A819B810E948408E82E8C819D810E94F7
:1011C0008408F82E8E819F810E948408F0E4DF9EBF
:1011D000A001112490E1E99E90011124242B282BD9
:1011E000E4E0FE9EB0011124262BF8012083CDB748
:1011F000DEB7E7E00C940E2F803223E0920708F16F
:10120000883E23E0920740F48F519340E4E09695A6
:101210008795EA95E1F70895803D27E0920718F455
:101220008C5D93400895883928E0920768F4885CC3
:10123000974074E0969587957A95E1F78D509C4F8D
:10124000089580E090E008958FEF93E008958C304A
:10125000910540F4A4E0880F991FAA95E1F7885DF5
:101260009C4F0895843F23E0920718F484529C4FCA
:101270000895811524E0920740F48657934FF4E0D7
:10128000880F991FFA95E1F7089580E998E008958D
:101290009C013695279525753575821B930B9C010E
:1012A0002373337396958795969587958373937378
:1012B000820F931F9C0154E0369527955A95E1F7CC
:1012C000280F391F2F703F7041E051E0249FC0016B
:1012D000259F900D349F900D1124892F08952D98EE
:1012E000882319F000002B9A02C000002B98000000
:1012F0002D9A000008952D9A000083B12D980000CA
:10130000829581700895CF93DF93D82F5C9A2D98A2
:101310005C98C8E08D2F80780E946F09DD0FC15066
:10132000C9F72D98DF91CF9108958F770E94830997
:101330000895CF93DF93D82FC8E08D2F80780E9437
:101340006F09DD0FC150C9F72D98DF91CF91089536
:10135000CF93DF932D98C8E080E0D82FDD0F0E9457
:101360007B098D0FC150C9F7DF91CF9108950E947D
:1013700095090E94A8095C9A0895A1E0B0E0E3EC09
:10138000F9E00C94F72E806869830E9483096981D3
:10139000862F0E9499095C9A2196E2E00C94132F03
:1013A000CF93C0917F05C827E82FF0E0EA58FA4FA5
:1013B000678589E70E94BD096C2F8DE30E94BD09F6
:1013C0006C2F82E40E94BD09CF91089586E20E94AD
:1013D000B7090895CF93DF93EC016C818CE10E94F3
:1013E000BD096D818DE10E94BD096E818EE10E9473
:1013F000BD096F8180E20E94BD09688581E20E947B
:10140000BD09698582E20E94BD096A8583E20E9466
:10141000BD096B8584E20E94BD096C8585E20E944E
:10142000BD096D858AE20E94BD096E858EE60E9427
:10143000BD096F858FE60E94BD09688980E70E941B
:10144000BD09698981E70E94BD096A8982E70E9416
:10145000BD09DF91CF910895CF92DF92EF92FF9275
:10146000CF93DF936B017C01C11488E3D8068CE92C
:10147000E8068CE1F80628F5C701B60120E836E950
:1014800048E950E00E94A62EE901689760E879E6F5
:1014900087E69FEF0E94822E6C0D7D1D8E1D9F1D85
:1014A000F2E0660F771F881F991FFA95D1F721E7A1
:1014B00032E040E050E00E94A62EF22EE32E80E4BF
:1014C00021C0C701B60120E03DE241E351E00E94A6
:1014D000A62EE901689760E073ED8EEC9EEF0E9406
:1014E000822E6C0D7D1D8E1D9F1D660F771F881F20
:1014F000991F21E732E040E050E00E94A62EF22E34
:10150000E32E80E66C2F6F71680F85E70E94BD099E
:101510006E2D86E70E94BD096F2D87E70E94BD09E9
:10152000DF91CF91FF90EF90DF90CF900895682FDB
:101530008DE60E94BD0908958F929F92AF92BF924F
:10154000CF92DF92EF92FF92CF93DF93D82F61E09B
:1015500089E00E94342A62E370E080E090E00E941B
:10156000712960E089E00E94342A62E370E080E043
:1015700090E00E94712983E00E94B7098093710571
:1015800084E00E94B7098093700560E086E00E94C5
:10159000BD0961E087E00E94BD096FE789E00E9414
:1015A000BD0965E08AE00E94BD0965E18BE00E940B
:1015B000BD0962E18CE00E94BD096DEF8DE00E94E3
:1015C000BD0960E08EE00E94BD09DD2319F08BE2C9
:1015D00091E008C020919D0533E1239FC0011124B3
:1015E000825C9E4F0E94EA096CE880E30E94BD097C
:1015F0006FE082E30E94BD0962E483E30E94BD09BB
:1016000080919E0587FF02C064E101C06AE084E327
:101610000E94BD096AE285E30E94BD096DE286E38E
:101620000E94BD0964ED87E30E94BD0960E088E384
:101630000E94BD0960E089E30E94BD09D11109C083
:10164000C0907F05D0908005E0908105F0908205E4
:1016500007C0C5E9CC2EC1ECDC2EED2CCEEDFC2E66
:10166000CAE38F2C9924AA24BB24682D8C2F0E94B6
:10167000BD09682D85E08C0F0E94BD09FE2CED2C64
:10168000DC2CCC24CF5FCE3361F76FEF83E40E9474
:10169000BD096FEF84E40E94BD096FEF85E40E94ED
:1016A000BD096FEF86E40E94BD09DD2311F066E0FD
:1016B00002C0609183058DE60E94BD0960E089E764
:1016C0000E94BD09609184058AE70E94BD0960E01F
:1016D00083E70E94BD0960E084E70E94BD09D11143
:1016E00009C060917B0570917C0580917D0590918A
:1016F0007E0504C060EC72E98DEE99E10E942C0A2F
:10170000DF91CF91FF90EF90DF90CF90BF90AF909F
:101710009F908F90089561E087E00E94BD0964E288
:101720008EE70E94BD0963E088E00E94BD0960E089
:1017300088E00E94BD0965E087E00E94BD0962E083
:1017400085E00E94BD0983E00E94B709809371057E
:1017500084E00E94B70980937005089583E00E9499
:10176000B7098093710584E00E94B70980937005E2
:1017700061E087E00E94BD096AE070E080E090E0EF
:101780000E9471290E948B0B00000895CF92DF9276
:10179000FF920F931F93CF93DF931F92CDB7DEB7C6
:1017A000082F162F8EE399830E94BD09F02EC02EBC
:1017B0009981D92E8C2D8F19811738F4F6016191FA
:1017C0006F018FE70E94BD09F5CF64E085E00E94BC
:1017D000BD0983E00E94B7098093710584E00E94EF
:1017E000B709809370050E944E2960936C05709331
:1017F0006D0580936E0590936F0569E087E00E9408
:10180000BD0981E0809373050F90DF91CF911F9107
:101810000F91FF90DF90CF9008950F931F930E9438
:10182000C60B80917305813099F40E944E29009176
:101830006C0510916D0520916E0530916F05601B50
:10184000710B820B930B603A76488140910548F307
:1018500080917305813031F46EE971E082EE95E09C
:101860000E943A2B1F910F9108950F931F9380911F
:101870007305823021F41092730581E020C08091BD
:1018800073058130D9F40E944E2900916C051091A6
:101890006D0520916E0530916F05601B710B820BF9
:1018A000930B613A76488140910540F061E087E012
:1018B0000E94BD091092730582E001C080E01F9173
:1018C0000F910895CF93DF93EC014AE050E06D2F24
:1018D00070E082EE95E00E94082C6EE282EE95E0C8
:1018E0000E940C2BBE0184E0769567958A95E1F7FE
:1018F0006F7077274AE050E082EE95E00E94082C56
:101900006EE282EE95E00E940C2BBE016F7077278D
:101910004AE050E082EE95E00E94082CDF91CF91E2
:101920000895D82FC0E0CD1780F45E9A64E670E089
:1019300080E090E00E9471295E9864E670E080E0AB
:1019400090E00E947129CF5FEECF6CE271E080E001
:1019500090E00E947129E6CF0F931F93CF93DF93FE
:10196000EC01062F15E0115051F0CE010E94033119
:10197000081741F0602FCE010E940B31F4CF82E0B6
:101980000E94910CDF91CF911F910F910895A0E0DB
:10199000B0E0EDECFCE00C94E92E482E562EC0E0B1
:1019A000D0E0612C712CE12CF12C00E010E0411012
:1019B0000CC06090D40586E4689E3001112459E182
:1019C000E52EF12C0AEB15E01EC091E049120FC084
:1019D0006090D405E6E46E9E30011124FBE16F0EA9
:1019E000711C49E2E42EF12C06E715E00CC082E000
:1019F000481209C028E1622E77247394EE24E39400
:101A0000F12C03ED15E043018C0E9D1E109275051F
:101A1000109274053401A62CA818B12CC3010196AC
:101A20006C01AE14BF04A8F4A00EB11E511006C084
:101A3000C3010E940331F501808305C0F501608177
:101A4000C3010E94AC0CF50180810E946106360141
:101A5000E2CFC301511018C0C3010E940331B82E58
:101A6000C6010E9403312B2D30E0322F2227282B74
:101A700080917405909175058217930779F4C0E001
:101A8000D0E05524539493CF3601609175050E94A0
:101A9000AC0C60917405C6010E94AC0CC05EDE4FB8
:101AA000C13E92E0D90708F482CF852DCDB7DEB7CD
:101AB000E0E10C94052F61E082E00E94C70C0895DC
:101AC00060E082E00E94C70C8091D305853020F051
:101AD0001092D3050E945B0D8091D3058093D405AD
:101AE000089561E080E00E94C70C61E081E00E94FF
:101AF000C70C089560E080E00E94C70C882351F075
:101B000060E081E00E94C70C882321F08091760577
:101B1000883349F00E94BF060E947A0681E00E9445
:101B2000DF060E94710D0895882319F06AEA71E0BA
:101B300002C06EEA71E082EE95E00E943A2B0895B1
:101B4000FF920F931F93CF93DF9369EC7BE082EEBC
:101B500095E00E94E62A40917B0550917C056091BA
:101B60007D0570917E052AE030E082EE95E00E94CE
:101B70000F2C63EB7BE082EE95E00E94E62A409119
:101B80007F0550918005609181057091820520E16B
:101B900030E082EE95E00E940F2C6DE97BE082EE52
:101BA00095E00E94E62A4AE050E06091830582EECB
:101BB00095E00E94372C67E87BE082EE95E00E947A
:101BC000E62A4AE050E06091840582EE95E00E94AA
:101BD000372C61E77BE082EE95E00E94E62AC5E8BB
:101BE000D5E0F12C8E0188818823A9F0FF2031F007
:101BF00061EB71E082EE95E00E94092B21964AE0AC
:101C000050E0F801608182EE95E00E94002CF39490
:101C1000F8E1FF12E7CF82EE95E00E94142B6BE50E
:101C20007BE082EE95E00E94E62A4AE050E0609177
:101C30009D0582EE95E00E94372C66E47BE082EE03
:101C400095E00E94E62AE0919E05E770F0E0EE0F35
:101C5000FF1FEE57FC4F6081718182EE95E00E947C
:101C60003A2B61E37BE082EE95E00E94E62A8091C8
:101C70009E058871883069F028F4811113C068E2EC
:101C80007BE00CC0803141F0883161F46CE07BE096
:101C900005C06CE17BE002C066E17BE082EE95E08E
:101CA0000E94282B68EF7AE082EE95E00E94E62AF7
:101CB00040917705509178056091790570917A058A
:101CC0002AE030E082EE95E00E940F2C6FED7AE082
:101CD00082EE95E00E94E62A8091BF0580710E9405
:101CE000940D66EC7AE082EE95E00E94E62A8091FF
:101CF000BF0580740E94940D6DEA7AE082EE95E053
:101D00000E94E62A8091BF0580720E94940D60E9CE
:101D10007AE082EE95E00E94E62A86E795E00E944E
:101D20001208AB01BC012AE030E082EE95E00E948F
:101D3000F12B6BE87AE082EE95E00E94E62A86E7D6
:101D400095E00E9412089B01AC0160E472E48FE010
:101D500090E00E94A62EBA01A9012AE030E082EEAE
:101D600095E00E94F12B68E87AE082EE95E00E940F
:101D7000282BCDB7DEB7E5E00C94102F8F929F9201
:101D8000AF92BF92CF92DF92EF92FF92811107C084
:101D90006FE77AE082EE95E00E94282B2FC090E05A
:101DA0000E94740724E630E040E050E00E94A62E36
:101DB000CA01B9012AE030E040E050E00E94A62EBE
:101DC00049015A016B017C012AE030E0B501A40110
:101DD00082EE95E00E94F12B6EE282EE95E00E9489
:101DE0000C2B2AE030E0B701A60182EE95E00E94BC
:101DF000F12B63E782EE95E00E944C2BFF90EF9071
:101E0000DF90CF90BF90AF909F908F9008951F93D9
:101E1000CF93DF9365E77AE082EE95E00E94E62AB1
:101E200080919F05813041F46CE57AE082EE95E087
:101E30000E94282B10E050C0823019F465E47AE04B
:101E4000F5CF843019F461E37AE0F0CF853091F773
:101E500066E27AE0EBCFC12FD0E0C930D1050CF4B7
:101E600041C068E3610F82EE95E00E940C2B6EE1A9
:101E70007AE082EE95E00E94E62ABE016F5F7F4F16
:101E80004AE050E082EE95E00E94D02B63E17AE0D8
:101E900082EE95E00E94E62AC156DA4FE981E032EF
:101EA00018F566E07AE082EE95E00E94E62A8981E4
:101EB000803130F06DE673E082EE95E00E94092BF0
:101EC00069816F7070E06F5F7F4F4AE050E082EE93
:101ED00095E00E94D92B1F5F80914805181708F4E0
:101EE000BACF0FC061E3BECFEF70F0E0EE0FFF1F7F
:101EF000EE56FC4F6081718182EE95E00E943A2B94
:101F0000EACF6BEE79E082EE95E00E94E62A8091BE
:101F1000B7050E94BE0E60ED79E082EE95E00E946A
:101F2000E62A8091B8050E94BE0E65EB79E082EE4C
:101F300095E00E94E62A8091B9050E94BE0E6AE9EA
:101F400079E082EE95E00E94E62A4091AF0550913B
:101F5000B0056091B1057091B2054115510561055B
:101F6000710539F12AE030E082EE95E00E940F2CF5
:101F700067E679E082EE95E00E94E62A8091B3055B
:101F80000E949907AB01BC012AE030E082EE95E0A7
:101F90000E940F2C63E479E082EE95E00E94E62A2D
:101FA0004AE050E06091B40582EE95E00E94372C43
:101FB00006C06AE379E082EE95E00E94282B6DE18D
:101FC00079E082EE95E00E94E62A6091B505709175
:101FD000B6054AE050E082EE95E00E94212C60E0D8
:101FE00079E082EE95E00E94E62A6091AE056034C9
:101FF00050F470E06F5F7F4F4AE050E082EE95E072
:102000000E94D92B06C067EF78E082EE95E00E942F
:10201000282B6AED78E082EE95E00E94E62A809116
:10202000AD0580FF03C063EB71E002C067EB71E0B8
:1020300082EE95E00E943A2B6DEB78E082EE95E01F
:102040000E94E62A8091AD0582700E94940D6EE98F
:1020500078E082EE95E00E94E62A8091AD058470DA
:102060000E94940D6FE778E082EE95E00E94E62AE8
:102070008091AD0588700E94940DDF91CF911F91E2
:1020800008950F931F93CF93DF93209145052F3F22
:10209000A9F56FEF75E082EE95E00E94E62A84E8EC
:1020A00093E00E94620C6EED75E082EE95E00E9476
:1020B000E62A80914605909147050E94620C6BEAE2
:1020C00075E082EE95E00E94282B68E875E082EECC
:1020D00095E00E94282B60E775E082EE95E00E9473
:1020E000282B6BE475E082EE95E00E94282B82EEAF
:1020F00095E00E94142B0E94070F68C012160CF086
:1021000065C0332727FD30958091480590E0821700
:1021100093070CF45BC066E375E082EE95E00E94E5
:10212000E62A60914505772767FD70954AE050E003
:1021300082EE95E00E94D92B6BE075E082EE95E08F
:102140000E94E62A10E008E2809149051817D0F5B0
:10215000C12FD0E0CC0FDD1FC65BDA4F288130E005
:1021600080914505992787FD909501972817390794
:1021700039F56BEB71E082EE95E00E94092B4AE0A5
:1021800050E0602F82EE95E00E94002C6FEB71E032
:1021900082EE95E00E94092BE981EF70F0E0EE0FEE
:1021A000FF1FEE56FC4F6081718182EE95E00E9428
:1021B000092B63EC71E082EE95E00E94092B0F5F22
:1021C0001F5FC2CF82EE95E00E94142BDF91CF916A
:1021D0001F910F910895FF920F931F93CF93DF9359
:1021E000C5E8D5E0F12C8E0188818823D1F165EC1A
:1021F00071E082EE95E00E94092B4AE050E06F2DDD
:1022000082EE95E00E94002C62ED71E082EE95E096
:102210000E94092B2196F801208130E0A0E1B7E26D
:102220000E94602E9B01AC01A0918405B0E00E9449
:102230006F2EAB01BC0180917B0590917C05A09134
:102240007D05B0917E05480F591F6A1F7B1F2AE04C
:1022500030E082EE95E00E940F2CF394F8E1FF123B
:10226000C2CFCDB7DEB7E5E00C94102F1092DF049B
:1022700085E6E0EEF4E0DF011D928A95E9F7089526
:10228000CF93C82F8F3719F0883009F045C0E091FF
:10229000DF04EE23D9F1E150E093DF04F0E0E052F7
:1022A000FB4F10826DE070E082EE95E00E945906CF
:1022B000C0E08091DF04C81760F4EC2FF0E0E0523A
:1022C000FB4F608170E082EE95E00E945906CF5F7F
:1022D000F0CF60E270E082EE95E00E9459066DE07A
:1022E00070E082EE95E00E945906C0E08091DF0424
:1022F000C81778F5EC2FF0E0E052FB4F608170E0FA
:1023000082EE95E00E945906CF5FF0CF67E082EE43
:1023100095E00E940C2B1DC08B3119F40E943611E0
:102320001AC08D30C1F08A30B1F08091DF0484365C
:1023300068F76C2F70E082EE95E00E945906E091FC
:10234000DF0481E08E0F8093DF04F0E0E052FB4F6A
:10235000C08380E001C081E0CF910895CF93C82F62
:102360000E944E296093C8047093C9048093CA04E4
:102370009093CB04C093DD04CC2329F040E051EED0
:1023800060E070E004C040E855E260E070E082EE9A
:1023900095E00E94962DCF9108959091CC04492FFD
:1023A0004F7050E0BA016F5F7F4F292F30E0E4E0BB
:1023B00035952795EA95E1F76217730759F0FA0109
:1023C000E353FB4F808381E0890F8F70907F892BCF
:1023D0008093CC0408956EE770E082EE95E00E9451
:1023E00059060895A3E1B1E0E8EFF1E10C94EA2E7B
:1023F000E5E8F5E0712C8191882321F0739428E1C0
:102400007212F9CF66ED71E082EE95E00E943A2BF0
:102410004AE050E0672D82EE95E00E94372C80E084
:102420000E949C0A0E948B0B8E010E5F1F4FC12CD5
:10243000D12C7601C39466246A945C2C0E944229B4
:102440004B015C012091840530E0A0E1B7E20E94DD
:10245000602E9B01AC01C701B6010E94822E209123
:102460007B0530917C0540917D0550917E05620F82
:10247000731F841F951F2091BB053091BC054091AF
:10248000BD055091BE05261737074807590718F4B0
:10249000F801608225C08C2D0E94D00961E070E0B7
:1024A00080E090E00E947129F80110820E94422988
:1024B000681979098A099B09643F71408105910572
:1024C00040F40E94E609F8019081981778F780831C
:1024D000EDCF50FE03C05D985E9A02C05D9A5E9893
:1024E0002FEFC21AD20AE20AF20A0F5F1F4F8FEFD4
:1024F000C816D104E104F10409F09FCFCE019395F1
:10250000FC01D82E7FEF68EC2E2F281B271510F02A
:1025100051E056C0DE01129651E02FEF41E03D91AF
:10252000321710F0322F01C0452F5F5F5F3F11F06F
:10253000232FF5CF4193242F30E0A1E0B0E0AC0F82
:10254000BD1FA20FB31F5C93413079F0DE01A20FD3
:10255000B31F5C93423049F0AFEFBFEFAC0FBD1F2C
:10256000A20FB31F6C934E3F78F6A2E0B0E0AC0F21
:10257000BD1FA20FB31F7C934D3F30F6A3E0B0E028
:10258000AC0FBD1FA20FB31F6C93BECF452F242FDE
:1025900030E0FC01E20FF31F6081AFEFB0E0AC0F61
:1025A000BD1FA20FB31F2C91621748F44150DC01EC
:1025B000A40FB11D2C9120836C934111E8CF5F5F74
:1025C000571520F3372D369520E0231770F4DC01E2
:1025D000A20FB11D4C91522F530FFC01E50FF11DBD
:1025E00050815C9340832E5FF0CFF5E8EF2EF5E04D
:1025F000FF2E8C01802F8D19871598F4F801C1905A
:102600008F014AE050E06C2D82EE95E00E94002C94
:102610006CE282EE95E00E940C2BF701C1927F01E3
:10262000E9CF82EE95E00E94142B81E0CD5EDE4F73
:10263000EFE00C94062F1F920F920FB60F92112409
:102640001F932F933F934F935F936F937F938F933A
:102650009F93AF93BF93CF93DF93EF93FF93C0917B
:102660008600D09187008091870490918804209102
:10267000A904211155C09E01281B390B8091BF056B
:102680009091C005A091C105B091C20585FD02C021
:1026900036952795253C49E03407B8F140910A0169
:1026A00050E060E070E02CE1B695A795979587958E
:1026B0002A95D1F70097A105B10521F481E090E0BA
:1026C000A0E0B0E084179507A607B707D8F480917B
:1026D0000A018F3FB9F040E080910A01481780F469
:1026E000842F90E0880F991FFC01E757FB4F208152
:1026F0003181FC01E55FFE4F318320834F5FECCFDA
:102700001092AA0410920A010BC02D3B82E03807F8
:1027100020F080910A018031D8F08FEF80930A0178
:10272000D0938804C0938704FF91EF91DF91CF91FC
:10273000BF91AF919F918F917F916F915F914F91D9
:102740003F912F911F910F900FBE0F901F901895E2
:1027500010910A0181E0810F80930A01C9010E9452
:10276000FC08E12FF0E0EE0FFF1FE757FB4F9183CE
:102770008083D6CF83E0809380008AE980938100B4
:102780008091BF0586FD05C08091810080648093A3
:1027900081008FEF9FEF9093890080938800809154
:1027A0006F00806280936F000895CF93DF930E9443
:1027B000600D8091D405843039F58FE00E94672A3E
:1027C000C1E0D0E0892B11F4C0E0D0E080E10E94AC
:1027D000672A892B19F082E090E002C080E090E047
:1027E0008C2B9D2B8230910539F08330910539F087
:1027F000019739F481E006C01092D40505C082E04B
:1028000001C083E08093D405DF91CF9108956F30AC
:1028100018F086958058089589E0689F802D1124CE
:102820000895A0E0B0E0E7E1F4E10C94F12EC82FA8
:102830000E944E29009138041091390420913A04E5
:1028400030913B046B017C01C01AD10AE20AF30A01
:102850009701860149E8C41643E1D406E104F10476
:1028600010F010923C046093380470933904809304
:102870003A0490933B042091A9048FEF820F823099
:10288000D8F5E0913C04EE2309F44EC1E13011F497
:1028900082E0B8C1E03108F034C181E08E0F80934E
:1028A0003C04F0E0E757FB4FC083803109F0ACC136
:1028B000EBE8F4E0213029F4A181A695A69580816A
:1028C00008C080819181A92FA695A695A695969579
:1028D0008795A03148F4B0E090E0AA0FBB1FA55F38
:1028E000BE4F11969C938E931092AA04329684E068
:1028F000E939F807F9F688C1233009F005C1E091FC
:102900003C04E11104C0CF3009F07EC10DC1E831B3
:1029100048F481E08E0F80933C04F0E0E857FB4FD1
:10292000C08372C1E83109F0ECC0C111EAC040E0D7
:1029300050E0ABE0CA01B3E0880F991FBA95E1F708
:10294000A49F9001A59F300D1124F901E757FB4F7B
:102950006081E1817E2F777075956795FC01EE0FA0
:10296000FF1FE55FFE4F71836083F901E657FB4F60
:10297000B081B695B695B695E181FE2FF295FF0F21
:10298000F07E6F2F6B2BE695E695E6957E2F7770A0
:1029900075956795FC01EE0FFF1FE35FFE4F718396
:1029A0006083F901E557FB4FB081B295B695B695B6
:1029B000B370C181DC2FDD0FDD0F6D2F6B2BC29546
:1029C000C695C695C370E281E170EE0FEE0F7E2FC3
:1029D0007C2B75956795FC01EE0FFF1FE15FFE4FA5
:1029E00071836083F901E357FB4FB081B695E181B4
:1029F000FE2FF795FF27F7956F2F6B2BE6957E2F10
:102A0000777075956795FC01EE0FFF1FEF5EFE4F27
:102A100071836083F901E257FB4FB081B295BF70BB
:102A2000E181FE2FF295F07F6F2F6B2BE295EF7017
:102A30007E2F777075956795FC01EE0FFF1FED5E99
:102A4000FE4F71836083F901E157FB4FB081BB1FDB
:102A5000BB27BB1FC181DC2FDD0F6D2F6B2BCC1F64
:102A6000CC27CC1FE281E370EE0F7E2F7C2B759577
:102A70006795FC01EE0FFF1FEB5EFE4F71836083D5
:102A8000F901EF56FB4FB081B695B695E181FE2F67
:102A9000F295FF0FFF0FF07C6F2F6B2BE695E695FD
:102AA0007E2F777075956795FC01EE0FFF1FE95E2D
:102AB000FE4F71836083F901EE56FB4F2081229512
:102AC000269527703181E32FEE0FEE0FEE0F6E2F5C
:102AD000622B732F72957695777075956795FC01CB
:102AE000EE0FFF1FE75EFE4F718360834F5F5F4F06
:102AF0004230510509F01ECF80919F0483FF109250
:102B0000AA0410923C0480C0243009F07DC060917A
:102B10003C0461110BC0C83AB1F4109275051092D3
:102B2000740588EA0E94610681E06CC0613019F486
:102B3000C093370404C0623031F4C09336048C2F44
:102B40000E9461065AC0E09136042E2F30E0220F19
:102B5000331F462F50E0C9010296841795073CF0B9
:102B6000633268F7FA01EA57FB4FC083E8CF2D5F65
:102B70003F4F8C2F90E0609174057091750542175E
:102B8000530749F4982F8827862797279093750530
:102B90008093740532C06817790769F5809137040E
:102BA000813049F5E13118F080E180933604F090EE
:102BB0003604CAE8D4E000E010E00F15D0F4FE01BE
:102BC0003197808190E0982F88272881822B63E0BD
:102BD000969587956A95E1F70E94FC08F801EE0F3B
:102BE000FF1FE55FFE4F918380830F5F1F4F22968B
:102BF000E4CF1092AA0410923C0480913C048823F4
:102C000019F08F5F80933C04CDB7DEB7E8E00C94F9
:102C10000D2FCF93DF93E82FF0E0E654FA4FE185D4
:102C2000E03150F4F894F0E0EE0FFF1FE55FFE4F47
:102C30008081918178945DC08EE08E0F8B3058F446
:102C4000F0E0E25FF10924E62E9FC0012F9F900D76
:102C500011240C964EC0E03F09F446C038F4E1312F
:102C600081F0E23191F0E03139F409C0ED3FB1F18A
:102C7000EE3FB9F1E13F79F180E092E03AC082E1C4
:102C800001C083E10E94902A34C08FE00E94672A2D
:102C9000C1E0D0E0892B11F4C0E0D0E080E10E94D7
:102CA000672A892B19F082E090E002C080E090E072
:102CB0008C2B9D2B8230910541F08330910541F0A2
:102CC0000197A9F086EA92E014C08CE090E011C070
:102CD00089E591E00EC086E090E00BC08AEF93E0BA
:102CE00008C08FEF93E005C080E090E002C084EF61
:102CF00093E0DF91CF910895A2E2B0E0E2E8F6E13F
:102D00000C94E72E9E012F5F3F4F80E1D9011D9269
:102D10008A95E9F764E072E082EE95E029A33AA390
:102D20000E943A2B0E94AE0B1D8A1E8A1F8A188EA3
:102D3000312C212C00E0812C912C540170E4472E81
:102D400071EE572E7DE9672E78E1772EE0E5CE2EE5
:102D5000E3ECDE2EE12CF12C84EF91E0A0E0B0E07A
:102D60008D8F9E8FAF8FB8A380EC91EDA8E9BBE16A
:102D7000898F9A8FAB8FBC8F80E491EEADE9B8E17B
:102D8000898B9A8BAB8BBC8B82EE95E00E944E2C8C
:102D9000892B09F4E1C082EE95E00E947B2C9C0116
:102DA00033272C32310509F442C0ACF4233231050B
:102DB00009F0ABC019821A821B821C821D821E82FE
:102DC0001F82188619861A861B861C861D861E86FB
:102DD0001F86188A60C02434310529F02335310557
:102DE00009F4B2C092C064E482EE95E00E940C2B1C
:102DF0002AE030E040E451EE6DE978E182EE95E0C2
:102E00000E949A2B6CE282EE95E00E940C2B2AE045
:102E100030E040EC51ED68E97BE182EE95E00E9404
:102E20009A2B6CE282EE95E00E944C2BADCF0F5FA7
:102E3000043009F0A9CF29813A814B815C81A8EE49
:102E4000B3E00E946F2E698B7A8B8B8B9C8B2D81CC
:102E50003E814F8158850E946F2E698F7A8F8B8FAC
:102E60009C8F29853A854B855C852D8F3E8F4F8FB2
:102E700058A32D853E854F8558890E946F2E6B0182
:102E80007C0160323EE473078105910530F462E312
:102E90008CE10E94BD0900E077CF603345E77407FD
:102EA0008105910510F462E2F3CF60345CE97507A7
:102EB0008105910510F466E2EBCF80E5C81683EC3E
:102EC000D806E104F10410F462E1E2CF90E6C916FD
:102ED0009AEED906E104F10410F465E1D9CFA0E738
:102EE000CA16A1E1DA06A1E0EA06F10410F461E0F5
:102EF000CFCFB0EACB16B6E8DB06B1E0EB06F104C3
:102F000010F463E0C5CF65E0C3CF10ED180F1A30A1
:102F100008F03ACFE1E0F0E0EC0FFD1F24E0029F63
:102F2000E00DF11D11242081318142815381AAE0FD
:102F3000B0E00E946F2E610F711D811D911D608395
:102F400071838283938320CF49885A886B887C88D9
:102F5000812C912C540118CF81149104A104B10447
:102F600089F4C301B2010E942C0A61E070E080E0A4
:102F700090E00E9471291D8A1E8A1F8A188E312CAA
:102F800022242A948D8D9E8DAF8DB8A18816990626
:102F9000AA06BB06D0F40E94E6092D893E894F8916
:102FA000588D280F311D411D511D2D8B3E8B4F8B90
:102FB000588F381608F4382E821508F4282E3FEF63
:102FC000831A930AA30AB30A56C0C301B20128EEBA
:102FD00033E040E050E00E94A62EBA01A9012AE0A9
:102FE00030E082EE95E00E94F12B6CE282EE95E0FB
:102FF0000E940C2B4AE050E0632D82EE95E00E9487
:10300000002C6CE282EE95E00E940C2B6D897E898B
:103010008F89988DA50194010E94A62EBA01A9015D
:103020002AE030E082EE95E00E94F12B6CE282EE25
:1030300095E00E940C2B4AE050E0622D82EE95E074
:103040000E94002C6CE282EE95E00E944C2B4C0C0E
:103050005D1C6E1C7F1C898D9A8DAB8DBC8D84157B
:103060009505A605B70520F449885A886B887C88A1
:10307000812C912C540129893A894B895C89283EFD
:1030800033404105510509F07FCEA296E2E10C9450
:10309000032FACE1B0E0EFE4F8E10C94F12E0E94D4
:1030A0004E296B017C0181E00E949C0A14E703E039
:1030B000198361E0CE0101960E940D0C0093730507
:1030C0000E948B0B6AEF70E080E090E00E94712913
:1030D00080917305833089F482EE95E00E944E2C36
:1030E000892B59F40E944E296C197D098E099F097C
:1030F0006038734C894C9140D8F2809173058330CD
:1031000009F44FC08FE70E9495090E94A80989839E
:10311000843511F083E05CC00E94A8091092460536
:10312000809347050E94A8092091460530914705E4
:10313000280F311D30934705209346050E94A809AA
:10314000809348050E94A80980934905813110F7B2
:10315000F12C0F2D10E08091490590E0880F991F08
:103160000817190740F40E94A809F801E65BFA4F16
:103170008083F394EECF80E7898361E0CE010196EE
:103180000E940D0C83E0809373050E948B0B62E319
:1031900070E080E090E00E94712980917305833097
:1031A00011F482E015C08FE70E9495090E94A809DA
:1031B0008983803509F0AECF0FE915E00E94A80998
:1031C000F80181938F01F5E00A3B1F07B9F781E011
:1031D0006C96E8E00C940D2F80914505992787FDAA
:1031E0009095A92FB92FFC013196EB30F10508F02D
:1031F00066C0EC5CFF4F0C941E2F62E778E082EE15
:1032000095E00E94282B84E893E00E94620C6AE516
:1032100078E082EE95E00E94282B65E378E082EE6C
:1032200095E00E94282B6BE078E082EE95E00E940A
:10323000282B6AEE77E082EE95E00E94282B6DEB5A
:1032400077E082EE95E00E94282B67E977E082EE36
:1032500095E00E94282B63E777E082EE95E00E94DC
:10326000282B6CE477E082EE95E00E94282B82EE1A
:1032700095E00E94142B0E94A00D21C06FE277E020
:103280001AC06AE077E017C065EF76E014C066ED1B
:1032900076E011C062E976E00EC06DE776E00BC023
:1032A00068E676E082EE95E00E94282B62E276E006
:1032B00002C06CE076E082EE95E00E94282B6AE086
:1032C00070E080E090E00E94712982EE95E00E941B
:1032D0004E2C892B29F082EE95E00E947B2CF5CFB5
:1032E0000895ACE1B0E0E7E7F9E10C94F12E90919C
:1032F00045059F3F09F023C1482F50E0FA013A9756
:10330000EF36F10508F00FC1E15CFF4F0C941E2F62
:1033100061E172E0A0C06DE172E082EE95E00E9492
:103320003A2B85E789838BE1EFE9F5E0DE01129620
:1033300001900D928A95E1F76CE1CE0101960E9411
:103340000D0C0E948B0B83E08093730568EC70E09A
:1033500080E090E00E94712980917305843009F02B
:10336000E2C08FE70E9495090E94A80989838535EC
:1033700009F0D9C06DEE74E082EE95E00E94282B32
:103380006FEC74E082EE95E00E94282B61EB74E014
:1033900096C065E372E082EE95E00E943A2B89E6E2
:1033A000898361E0CE0101960E940D0C0E948B0B77
:1033B00083E08093730568EC70E080E090E00E9409
:1033C000712980917305843009F0ADC08FE70E94A8
:1033D00095090E94A80989838E010E5F1F4F7E0107
:1033E0004DE1E40EF11C0E94A809F80181938F01C0
:1033F000EE15FF05C1F78BE1FE013296AFE9B5E0AE
:1034000001900D928A95E1F78981893409F08BC08A
:1034100063E974E082EE95E00E94282B65E774E092
:1034200082EE95E00E94282B67E574E048C06FE4C7
:1034300072E082EE95E00E943A2B8EEF8093450574
:1034400072C080528750805390914805981708F0B9
:1034500066C06EE572E082EE95E00E943A2B63C092
:1034600084E18093450560E274E029C085E18093A2
:10347000450569EE73E023C086E18093450562EB64
:1034800073E01DC087E18093450568E673E017C0CF
:1034900088E18093450567E573E011C089E1809379
:1034A000450563E473E00BC08AE1809345056EE255
:1034B00073E005C08BE18093450566E073E082EE22
:1034C00095E00E94282B2FC06CEE72E082EE95E012
:1034D0000E94282B8091AD0591E01DC066ED72E041
:1034E00082EE95E00E94282B8091AD0592E013C0FA
:1034F00061EC72E082EE95E00E94282B8091AD0590
:1035000094E009C066EA72E082EE95E00E94282B02
:103510008091AD0598E089278093AD058FEF80936A
:1035200045050E94411082EE95E00E944E2C892BA9
:1035300009F45BC182EE95E00E947B2CF4CF0E94DF
:103540004011882309F451C18091DF04811104C026
:103550008FEF8093450541C140E050E060E070E0AE
:1035600080EE94E00E94952F40914505042F11278D
:1035700007FD1095212F312FF8013197EB31F1051F
:1035800008F01BC1E255FF4F0C941E2F552747FD35
:1035900050952091480530E0241735070CF40DC1F3
:1035A0008B019C01015011092109310900321105DB
:1035B0002105310558F0C0904905EBE4F5E0F12C08
:1035C000D12CA8E2EA2E415051090FC0FA01E15670
:1035D000FA4F61506083D9C0DF0111972C9130E020
:1035E0002417350729F0F3943296FC10F5CFCBC0A1
:1035F0000E2D10E020E030E00617170728073907E6
:1036000041F42081DA01A156BA4F11962C93DD24A2
:10361000D394E394E8CF6F3F71058105910511F0D4
:1036200008F0CBC06093B705B0C06F3F710581054E
:10363000910511F008F0C1C06093B805A6C06F3FB6
:1036400071058105910511F008F0B7C06093B905C7
:103650009CC02091E00420622037E9F440E050E073
:1036600060E070E081EE94E00E94952F9B01AC0138
:10367000DC01CB010197A109B1090897A105B105AA
:1036800008F0AEC0A4EDB0E30E946F2E6A5E7C4AE3
:103690008A46954E24C02636E9F440E050E060E0CA
:1036A00070E081EE94E00E94952F9B01AC01DC015B
:1036B000CB010197A109B1090797A105B10508F050
:1036C0008FC0A8EAB1E60E946F2E645E7C438E46EE
:1036D000944E05C0611571058105910579F08B0146
:1036E0009C010054114E2D4938410138F0EF1F075D
:1036F000FAEF2F07F2E03F0708F05FC06093AF05D5
:103700007093B0058093B1059093B2053EC06F3FB2
:1037100071058105910511F008F04FC06093B30564
:1037200034C08B019C0101501109210931090F3F5F
:1037300011052105310508F040C06093B40525C08E
:103740008B019C01045C1940210931090D344DE1C4
:1037500014072105310528F47093B6056093B5056B
:1037600014C0611571058105910521F48FEF8093D7
:10377000AE050BC06134710581059105F0F461500F
:103780006093AE0502C0DD20C1F08091DE0481119E
:103790001AC080917F0590918005A0918105B0911C
:1037A00082050196A11DB11D80937F059093800530
:1037B000A0938105B093820506C060E772E082EEB7
:1037C00095E00E943A2B0E9436118FEF80934505B9
:1037D0006AE082EE95E00E944C2B0E94411005C0E9
:1037E00061E070E080E090E07ACF6C96E8E00C94C5
:1037F0000D2F6AE572E082EE95E00E94282B62E4CC
:1038000072E082EE95E00E94282B82EE95E00E9405
:103810004E2C892B31F082EE95E00E947B2C0E9489
:1038200071190E944918823029F0833051F46DE0FB
:1038300072E002C064E272E082EE95E00E94282B02
:1038400008958FEF809345051092DE040E94411089
:10385000809145058E3F69F082EE95E00E944E2CE6
:10386000892BB1F382EE95E00E947B2C0E947119A6
:10387000EFCF08950F931F93109145051F3F09F057
:10388000D2C0893409F457C000F5883309F469C0FF
:1038900058F4803309F477C008F061C08B3109F423
:1038A00040C08132B1F1B9C0813409F487C030F42D
:1038B000893309F466C0803461F1AFC0823409F401
:1038C0008EC0863409F448C0A8C0823609F487C087
:1038D00078F4883531F128F48235C1F18335E1F08F
:1038E0009CC08A3509F494C0813609F467C095C03C
:1038F000823761F128F4863679F18936E1F08DC09E
:10390000883779F08A3709F483C0833709F085C096
:1039100003C061E172E015C00E94710D6EE872E0B3
:1039200004C00E947A0D68EA72E082EE95E00E947F
:103930003A2B8EEF70C00E947A060E94BF0667EC99
:1039400072E082EE95E00E943A2B67C081E00E940F
:10395000DF0660EE72E0F5CF0E94EB105EC0805390
:103960005AC06AEF71E082EE95E00E94282B909198
:103970009E0588E0890F8871977E892B80939E052C
:103980001AC089E048C067EE71E082EE95E00E94BF
:10399000282B8091BF059091C005A091C105B091E1
:1039A000C20520E182278093BF059093C005A093B4
:1039B000C105B093C205109345052FC061ED71E0BC
:1039C00082EE95E00E94282B8091BF059091C00562
:1039D000A091C105B091C20540E4842710C060ECFD
:1039E00071E082EE95E00E94282B8091BF059091B6
:1039F000C005A091C105B091C20520E28227809345
:103A0000BF059093C005A093C105B093C20502C045
:103A10000E94F91B8FEF80934505809145058E3FED
:103A200009F0D4C0DDC00E944011882309F4D8C039
:103A30008091DF04811104C08FEF80934505C6C0DB
:103A400040E050E060E070E080EE94E00E94952F4E
:103A500000914505112707FD1095212F312FF80101
:103A60003197E930F10508F0B4C0E753FF4F0C94EB
:103A70001E2F8B019C010154114E2D4938410F37E7
:103A8000104F2A4F324008F0A4C060937B0570931A
:103A90007C0580937D0590937E0577C060937F05BC
:103AA00070938005809381059093820581E08093D7
:103AB000DE046BC0683071058105910508F089C08E
:103AC0006093830562C08B019C010150110921099B
:103AD00031090A3011052105310508F07AC06093DB
:103AE000840553C061EB71E080EE94E00E94CF301A
:103AF00010E0009799F00E94A930009779F01831F2
:103B000030F4E12FF0E0EA58FA4F87871F5F61EB4E
:103B100071E080E090E00E94CF30EBCF1831A8F543
:103B2000E12FF0E0EA58FA4F17861F5FF7CF6530B4
:103B300071058105910508F04CC060939D0525C075
:103B40008B019C0101501109210931090630110531
:103B500021053105F0F520919E05287F262B209325
:103B60009E0513C08B019C010150110921093109E7
:103B70000115124C2140310560F560937705709373
:103B800078058093790590937A058091DE04811100
:103B900013C080917F0590918005A0918105B0911F
:103BA00082050196A11DB11D80937F05909380052C
:103BB000A0938105B09382050E9436118FEF809308
:103BC00045056AE082EE95E00E944C2B0E94EC18BD
:103BD00007C060E772E082EE95E00E943A2BECCFDE
:103BE0001F910F9108958FEF809345051092DE0489
:103BF0000E94EC18809145058E3F69F082EE95E0B9
:103C00000E944E2C892BB1F382EE95E00E947B2C12
:103C10000E943A1CEFCF6AE070E080E090E00E94E2
:103C2000712982EE95E00E944E2C892B29F082EEBC
:103C300095E00E947B2CF5CF0895CF93C82F682F75
:103C400082EE95E00E94A82C90916A059C279093A3
:103C50006A05CF910895A1E0B0E0E1E3FEE10C94A4
:103C6000F72E99830E941D1E9981892F0E941D1E87
:103C70002196E2E00C94132F1F93CF93DF93182F1C
:103C8000EB0110926A0565EB70E082EE95E00E9410
:103C9000590662E670E082EE95E00E945906812F97
:103CA0000E941D1ECE010E942B1EDF91CF911F91FD
:103CB000089560916A0582EE95E00E94A82C08950F
:103CC000A1E2B0E0E6E6FEE10C94F32E7B018A016E
:103CD0008C3009F452C108F040C0863009F4BCC0F1
:103CE00018F5833009F491C070F4813009F472C082
:103CF000823009F047C26BE170E082E00E943C1E16
:103D00000FE915E078C0843009F487C0853009F0E8
:103D100039C26091490570E0660F771F85E00E9407
:103D20003C1E0AE415E086C0893009F4A7C070F48F
:103D3000873009F49BC0883009F024C261E070E04C
:103D400088E00E943C1E8091D40522C28A3009F48A
:103D5000CAC08B3009F4F1C015C28A3609F474C1A7
:103D6000D8F4873609F439C138F4853609F40DC121
:103D7000863609F41EC106C2883609F436C1893672
:103D800009F000C261E070E089E60E943C1E0E94DA
:103D90007A060E94BF06F4C18D3609F4D3C138F407
:103DA0008B3609F490C18C3609F499C1EBC18E367B
:103DB00009F4DBC1873C09F0E5C161E070E087EC04
:103DC0000E943C1E81E00E941D1E0E94591E1092FE
:103DD0006B05E2C169E270E081E00E943C1E06E7EB
:103DE00015E0F80181918F010E941D1EF5E00F3949
:103DF0001F07B9F7CFC1F80181918F010E941D1EE5
:103E0000F5E00A3B1F07B9F7C5C161E070E083E048
:103E10000E943C1E0E944918BBC161E070E084E032
:103E20000E943C1E81E00E941D1E0E94591E0E949D
:103E30007C16B2C18091490590E0880F991F9801C6
:103E40002A5435402817390708F0A4C1F801819198
:103E50008F010E941D1EEECF62E070E086E00E949E
:103E60003C1E84E893E00E942B1E94C161E070E048
:103E700087E00E943C1E809148058AC186E68983BE
:103E800061E0CE0101960E940D0C0E948B0B83E035
:103E90008093730568EC70E080E090E00E947129E7
:103EA000809173058430D9F48FE70E9495090E94B0
:103EB000A8098983863469F460E270E089E00E9491
:103EC0003C1E10E20E94A8090E941D1E1150D1F74D
:103ED00061C161E070E089E00E943C1E51C161E077
:103EE00070E089E052C169E170E08AE00E943C1E06
:103EF0001092BA05209172058091BF059091C0057E
:103F0000A091C105B091C205222311F0806801C0C3
:103F10008F778093BF059093C005A093C105B093A0
:103F2000C2050AEB15E0F80181918F010E941D1E68
:103F3000F5E0033D1F07B9F72DC161E270E08BE0AA
:103F40000E943C1E8091AA048F3F39F08091AA0400
:103F500091E0980F9093AA0402C08091AA040E9455
:103F60001D1E10E0812F0E9409160E9427090E9441
:103F70002B1E1F5F1031B1F70DC161E070E08CE0C6
:103F80000E943C1E8091D30503C161E070E085E68C
:103F90000E943C1E89E2E816F10409F0F8C0D8013D
:103FA000E6E7F5E08D91819385E0EF39F807D1F7E9
:103FB000E7C061E070E086E60E943C1EEBE1EE1691
:103FC000F10409F0E4C0D801EFE9F5E08D918193A7
:103FD00085E0EA3BF807D1F7D3C061E070E087E6FF
:103FE0000E943C1E0E94710DCBC061E070E088E62B
:103FF0000E943C1E85E789838BE1EFE9F5E0DE0155
:10400000129601900D928A95E1F76CE1CE0101962E
:104010000E940D0C0E948B0B83E08093730560E27D
:1040200073E080E090E00E947129809173058430F4
:1040300009F0ADC08FE70E9495090E94A809898305
:10404000853509F0A4C09CC061E070E08AE60E945A
:104050003C1E89E6898361E0CE0101960E940D0C29
:104060000E948B0B83E08093730560E273E080E035
:1040700090E00E94712980917305843009F087C017
:104080008FE70E9495090E94A80989838E010E5F1F
:104090001F4F7E01EDE1EE0EF11C0E94A809F80110
:1040A00081938F01EE15FF05C1F78BE1FE0132967A
:1040B000AFE9B5E001900D928A95E1F789818934E5
:1040C00009F065C05DC061E070E08BE60E943C1EB7
:1040D000F80180818093D4050E947A0D51C061E07F
:1040E00070E08CE60E943C1EF0E2EF16F10461F4F1
:1040F00087E6898380E2F801DE01129601900D9235
:104100008A95E1F761E203C087E4898361E0CE012B
:1041100001960E940D0C0E948B0B83E08093730527
:104120006CE474E080E090E00E9471298091730556
:10413000843069F58FE70E9495090E94A8098734A9
:1041400031F51EC061E070E08DE60E943C1E89E101
:10415000E816F104E1F4D801EAEBF5E08D918193E2
:1041600085E0E33DF807D1F70BC061E070E08EE633
:104170000E943C1EF80180818093D3050E945B0D54
:1041800081E006C061E070E08AEC0E943C1E80E0A5
:104190000E941D1E0E94591EA196E6E00C940F2F4E
:1041A000A0E0B0E0E6EDF0E20C94F12ECAECD3E032
:1041B00014E606E035E0F32E44E0E42E53E0D52E7D
:1041C00062E0C62E82EE95E00E944E2C892B09F407
:1041D0009BC082EE95E00E947B2C282F80933504B3
:1041E0004091340450E04730510560F7FA01EE5237
:1041F000FF4F0C941E2F853B29F781E080933404F8
:10420000E1CF823609F07DC0C0923404DBCF8093C9
:10421000330480933204D0923404D4CF9C013327EA
:104220003093310420933004909132049827909376
:104230003204E0923404C6CF382F22274091300454
:1042400050913104242B352B3093310420933004CA
:1042500090913204982790933204F09234042536DA
:10426000310508F4AFCF61E070E08CEC0E943C1E99
:1042700081E00E941D1E0E94591E43C020912E0401
:1042800030912F04F901E653FC4F80839091320462
:10429000982790933204C901019690932F0480933C
:1042A0002E0420913004309131048217930708F4D2
:1042B00089CF0093340486CF8091320482130BC0DF
:1042C00060912E0470912F044AEC53E080913304E6
:1042D0000E94601E0DC062E070E08BEC0E943C1EEC
:1042E000809133040E941D1E80916A050E941D1E4C
:1042F000FE01812F11928A95E9F710922F041092F6
:104300002E04109234045ECFCDB7DEB7E8E00C94F3
:104310000D2F81E080936B0580916B05882349F018
:1043200082EE95E00E944E2C892BB1F30E94D020A2
:10433000F3CF0895AAE2B0E0E0EAF1E20C94EF2EA8
:104340000E9442296B017C0181E00E949C0A82EE5E
:1043500095E00E944E2C892B29F082EE95E00E9478
:104360007B2CF5CF5E9811E072E6B72EE9E2AE2E17
:1043700003E00E9442296C197D098E099F09693C5E
:10438000710581059105D0F11123C1F10E944229E7
:104390006B017C015D9A80ED97E00E94AE07B982C7
:1043A000E6E7F5E0DE0112968A2D01900D928A95DE
:1043B000E1F76AE2CE0101960E940D0C5D9880E063
:1043C00090E00E94AE07009373050E948B0B62E39E
:1043D00070E080E090E00E94712980917305843044
:1043E00061F4009373058FE70E9495090E94A80964
:1043F00011E0823419F410E001C011E08EE00E9457
:10440000672A892B81F411E00EC05E9A5D9A82EED4
:1044100095E00E947B2C8D309105A9F05CF40A9701
:1044200091F05E985D9882EE95E00E944E2C892B6B
:1044300061F79FCF8332910579F08234910589F736
:104440000E948921EECF62EB71E082EE95E00E943E
:10445000282B0E94F31DE5CF0E947C16E2CF8F929D
:104460009F92AF92BF92CF92DF92EF92FF921F93F3
:10447000CF93DF938EE00E94672A892B09F089C0D1
:1044800068EC70E080E090E00E94712980E090E0AC
:104490000E94AE070E9442294B015C016B017C0126
:1044A00080ECC80E82E1D81EE11CF11C0E9442295A
:1044B0006C157D058E059F0530F48EE00E94672AFD
:1044C000892BA1F364C08EE00E94672A892B09F032
:1044D0005EC080ED97E00E94AE070E9442296B010A
:1044E0007C01D0E0C1E088E4880E86E2981EA11C21
:1044F000B11C11E08EE00E94672A892B21F58C14F3
:104500009D04AE04BF0430F480ED97E00E94AE0736
:10451000D1E0F0CF0E9442296C197D098E099F09D4
:10452000693C71058105910528F30E9442296B01C0
:104530007C01C12719F080ED97E002C080E090E097
:104540000E94AE07D7CF80E090E00E94AE07DD2347
:10455000B9F08091D30590E0019665E070E00E948B
:10456000922E8093D3050E945B0D0E94D5130E946A
:104570007A0D64EF71E080E090E00E94712909C03B
:1045800080E00E94DF060E94F2110E94710D0E94DD
:104590009A21DF91CF911F91FF90EF90DF90CF9004
:1045A000BF90AF909F908F900895CF92DF92EF923F
:1045B000FF9280E00E94F8070E94CF0761E089E047
:1045C0000E94FB2960E089E00E94342A61E086E0D5
:1045D0000E94FB2961E085E00E94FB2960E08EE0FB
:1045E0000E94FB2960E08FE00E94FB2961E08FE0E0
:1045F0000E94342A60E080E10E94FB2961E080E1B2
:104600000E94342A60E088E00E94FB2961E088E093
:104610000E94342A61E081E10E94FB2960E081E18F
:104620000E94342A0E949F0740E052EC61E070E053
:1046300082EE95E00E94962D0E94D5130E947A0D7D
:104640000E94BA138FEF8093AA040E94E407789423
:104650000E9442296B017C018091AA048F3F59F48A
:104660000E9442296C197D098E099F09603D77409F
:104670008105910588F380ED97E00E94AE0761E027
:104680008EE00E94342A5E9A82EE95E00E944E2CC3
:10469000892B29F082EE95E00E947B2CF5CF6DEFFF
:1046A00072E082EE95E00E94092B84E893E00E947C
:1046B000620C64E173E082EE95E00E94092B4AE00F
:1046C00050E064E070E082EE95E00E94D92B62E356
:1046D00070E080E090E00E94712982EE95E00E94F7
:1046E0004E2C04970CF182EE95E00E947B2C8234D4
:1046F0009105D1F482EE95E00E947B2C8E349105D9
:1047000099F482EE95E00E947B2C8434910561F44B
:1047100082EE95E00E947B2C819731F480E090E05E
:104720000E94AE070E949A2140917705509178052A
:104730006091790570917A05DB01CA010197A109A1
:10474000B1090497A105B10568F44093A904433069
:1047500029F440EA56E861E070E004C040E052EC21
:1047600061E070E082EE95E00E94962D0E942F227B
:104770005E9880E090E00E94AE070E94BA1310920B
:10478000C5048091BF0583FF11C080918B058823EC
:1047900051F080919205882331F08091990588230A
:1047A00011F087E001C085E08093C50480E00E949D
:1047B0009C0A8091C6040E94D0090E948B0B109223
:1047C0003F0410923E0410923D04F12C8091D405D8
:1047D0008F15B0F062E370E080E090E00E947129F4
:1047E00080ED97E00E94AE0762E370E080E090E029
:1047F0000E94712980E090E00E94AE07F394E6CF1A
:1048000080919E0584FF08C0982F987181E09831AF
:1048100009F080E00E94AE118FE00E94F807FF903F
:10482000EF90DF90CF900895EF92FF920F931F9338
:10483000CF93DF938C016EE770E082EE95E00E94EB
:104840005906E801F12CF0E2EF2E8E0188818D5798
:10485000823048F46DE770E082EE95E00E945906E0
:1048600088818E2588832196F801608182EE95E00B
:104870000E94A82CF394F9E0FF12E7CF6EE770E0F6
:1048800082EE95E00E945906CDB7DEB7E6E00C94C3
:104890000F2FA9E0B0E0EFE4F4E20C94F72E909132
:1048A000C70491110EC09EEF99838A836B8350E0F9
:1048B000559547954C832D83198618861F821E8235
:1048C0002EC04091CC04842F90E0B4E0959587955C
:1048D000BA95E1F7242F2F7030E08217930719F172
:1048E0008DEF89831B82FE01349650E0842F90E087
:1048F000A4E095958795AA95E1F7242F2F7030E0D5
:104900008217930749F0DC01A353BB4F8C9181932D
:10491000405F5F5F563051F74093CC045A83CE011D
:1049200001960E9414248091C70490E0019666E0ED
:1049300070E00E94922E8093C7042996E2E00C94C6
:10494000132FA0E0B0E0E7EAF4E20C94F02E6C0143
:104950006EE770E082EE95E00E9459068601E12C38
:10496000F12CC0E0D0E030E2B32EF801608183E8A2
:10497000860F823078F46DE770E082EE95E00E9459
:104980005906F80160816B2570E082EE95E00E9487
:10499000590604C082EE95E00E94A82CE114F104AF
:1049A00059F0F80180819E01280F311DC901C92FDE
:1049B000DD27C80FD91FDD273FEFE31AF30A89E08F
:1049C000E816F10459F028E0E216F10421F48C2FE6
:1049D0008095F60180870F5F1F4FC7CFCDB7DEB739
:1049E000E9E00C940C2FA9E0B0E0E9EFF4E20C94BC
:1049F000F72EE82F362F8091C70490E0019664E2ED
:104A000070E00E94922E8093C70458E9598350E1C8
:104A10005A83813089F048F08230B9F08330D9F47C
:104A20008B8381EF8C833D8319C085E08B8381EF7D
:104A30008C832F5F2D8312C08B8381EF8C8384E660
:104A4000489FA00111245D8309C084E08B8381EF1E
:104A50008C83ED8303C00E94EB1104C0CE0101964C
:104A60000E94A1242996E2E00C94132FA2E0B0E06A
:104A7000ECE3F5E20C94EC2E182F762E2A83498372
:104A80000E944E296B017C018091DD048090C80456
:104A90009090C904A090CA04B090CB042A814981A7
:104AA0008823C1F0D701C60188199909AA09BB0951
:104AB0004C015D0191EE89169EE29906A104B104B4
:104AC00020F1241708F4422F202F672D812F0E94F8
:104AD000F32413C0D701C60188199909AA09BB0993
:104AE0004C015D0191E3891695E79906A104B10493
:104AF00060F0672D812F0E944924C092C804D09293
:104B0000C904E092CA04F092CB042296EDE00C9422
:104B1000082FA2E2B0E0EFE8F5E20C94ED2E8CE075
:104B20000E94B70981110DC06CE173E082EE95E03F
:104B30000E943A2B5E9A80E00E949C0A0E948B0B96
:104B40005E9882EE95E00E944E2C892B01F182EE58
:104B500095E00E947B2C9091A904992319F00E9462
:104B60001114EFCF40913E0450E09A012F5F3F4F68
:104B70002F71332760913F0470E02617370709F340
:104B8000FA01E75BFB4F808320933E04DACF8091EC
:104B90007305843009F086C00E944E2961157105A5
:104BA0008105910549F06093B7047093B804809330
:104BB000B9049093BA040CC081E090E0A0E0B0E0AA
:104BC0008093B7049093B804A093B904B093BA0447
:104BD0008091AD049091AE0481609093AE04809377
:104BE000AD0483E0809373058FE70E94950909E681
:104BF00014E00E94A809F80181938F01F4E00237C4
:104C00001F07B9F72091720480916904982F9227A9
:104C100096FF3BC090E4922790937204982F98736C
:104C20009833F1F410E0212F30E08091690487700F
:104C300090E0821793074CF11F5F20919E05812F12
:104C400090E0FC01E759FB4F24FF04C080810E94E3
:104C5000CD11E9CF608182EE95E00E94A82CE3CFD0
:104C60008F7399F480916A048093B60480916B04E9
:104C70008093B40480916C048093B30480916F049A
:104C800090E09093AC048093AB0480913D0481301C
:104C900019F482E080933D0480913D04833011F447
:104CA00010923D040E944E296B017C018091AF045B
:104CB0009091B004A091B104B091B2040097A10505
:104CC000B105C9F0A7019601281B390B4A0B5B0BF4
:104CD000DA01C901883B9B40A105B10560F00E9443
:104CE000E6098093B5041092AF041092B0041092BC
:104CF000B1041092B2048091BB049091BC04A091C5
:104D0000BD04B091BE0446015701881A990AAA0A47
:104D1000BB0A86E795E00E94120886169706A80649
:104D2000B90608F4B1C0C092BB04D092BC04E092B2
:104D3000BD04F092BE040E9457068091AA048830F8
:104D4000A0F08091BF059091C005A091C105B091E0
:104D5000C2055CE1B695A795979587955A95D1F7C9
:104D6000892B8A2B8B2B09F0B8C18091AA048F5F05
:104D70008093AA048091B7049091B804A091B904DB
:104D8000B091BA040097A105B105F1F0C81AD90A8B
:104D9000EA0AFB0A86E795E00E9412086C157D0579
:104DA0008E059F0508F00FC18091BF0584FD04C0EA
:104DB00080ED97E00E94AE071092B7041092B804FD
:104DC0001092B9041092BA0490917204907C90935E
:104DD000720450913E0480913F0420913D04581785
:104DE00009F40EC1223009F00BC19058909372045F
:104DF000E0919E05E770F0E0E658FC4F6081693075
:104E000008F0E6C0615040E04613E4C080933F04E0
:104E100087E3840F90917204892B809372044093EE
:104E2000400483E080933D045D9A10918305809156
:104E3000C504811132C18091BF0582FD3AC1812F25
:104E40000E94970A8091C6040E94D009E0919E05B5
:104E5000E770F0E0E658FC4F608182E794E00E9442
:104E6000C60B8091BF0582FD2DC1E091C604EF5FA6
:104E7000E093C604E83109F42DC1F0E0EA58FA4F96
:104E80008785882309F426C10E94350C813069F595
:104E900080919E05887149F18091AD049091AE0496
:104EA000880F991F9093AE048093AD0483E08093A4
:104EB00073050E948B0B0E944E296093AF04709380
:104EC000B0048093B1049093B204672B682B692BD4
:104ED00061F481E090E0A0E0B0E08093AF049093B3
:104EE000B004A093B104B093B20480919E0584FFF6
:104EF0001FC08091AD049091AE048E7F0E9448093E
:104F0000182F6091AB048091B6040E940714482FBB
:104F1000612F8091B50449A30E9407140091D40524
:104F2000282F49A16091B3048091B4040E943625D2
:104F30005D988091C3048130C1F018F08230B1F1E6
:104F4000D9C08EE00E94672A892B09F0D3C081E086
:104F50008093C3040E9442296093BF047093C004ED
:104F60008093C1049093C204C5C08EE00E94672A5A
:104F7000892B31F50E944229C090BF04D090C00413
:104F8000E090C104F090C2046C197D098E099F095C
:104F9000693E73408105910508F4ACC082E08093BE
:104FA000C30480ED97E00E94AE07A4C08EE00E948B
:104FB000672A892B09F49EC080E090E00E94AE072A
:104FC0001092C30497C080E090E00E94AE07FCCE30
:104FD00068E019CF851709F419CF4F5F242F30E00F
:104FE00090E0F901EE58FB4FDC01A75BBB4F7C91D1
:104FF0007083F901E05CFB4F708301968F7104CFE1
:105000002430B1F42091400481E494E0A3E7B4E0BB
:10501000FC013E2F381B321718F431913D93F9CF24
:1050200087E3820F90917204892B80937204F9CEEA
:105030008091C304823051F49160909372045E9A1F
:105040008E010F5F1F4FF12CB80110C05E98809148
:105050003D04811103C081E080933D0480913D04B3
:10506000833071F784E080933D04EACF8F2D69A3EC
:105070007AA30E940916F801819391938F01F3940A
:1050800069A17AA1F0E1FF12F1CF80919E0543E77B
:1050900054E087700E949708C7CE112309F4CBCE45
:1050A0009091C40421E0290F2093C4049813C3CE27
:1050B0001DC08FE00E94672A892B09F0C0CE5E9A3E
:1050C00017E0BDCE8FE00E94672A892B09F0CDCE74
:1050D0005E98CBCE1092C604D7CE8091AA048830B9
:1050E00009F45E9A89E08093AA04CECE1092C4049B
:1050F0001150A1CEA296ECE00C94092F8230E8F476
:10510000E82FF0E0EE0FFF1FEB52FA4F7183608340
:10511000813041F0809169008C7F842B80936900FD
:10512000E89A089580916900440F551F440F551F58
:10513000837F842B80936900E99A08951F920F92D0
:105140000FB60F9211242F933F934F935F936F935A
:105150007F938F939F93AF93BF93EF93FF93809130
:10516000D5059091D605892B29F0E091D505F091D0
:10517000D6050995FF91EF91BF91AF919F918F91C6
:105180007F916F915F914F913F912F910F900FBE43
:105190000F901F9018951F920F920FB60F92112427
:1051A0002F933F934F935F936F937F938F939F932F
:1051B000AF93BF93EF93FF938091D7059091D8055C
:1051C000892B29F0E091D705F091D8050995FF9139
:1051D000EF91BF91AF919F918F917F916F915F916F
:1051E0004F913F912F910F900FBE0F901F901895E8
:1051F0001F920F920FB60F9211242F933F938F930C
:105200009F93AF93BF938091DA059091DB05A091B6
:10521000DC05B091DD053091D90523E0230F2D3752
:1052200020F40196A11DB11D05C026E8230F0296AA
:10523000A11DB11D2093D9058093DA059093DB055C
:10524000A093DC05B093DD058091DE059091DF052C
:10525000A091E005B091E1050196A11DB11D8093DB
:10526000DE059093DF05A093E005B093E105BF91C3
:10527000AF919F918F913F912F910F900FBE0F9003
:105280001F9018952FB7F8946091DA057091DB059F
:105290008091DC059091DD052FBF08953FB7F8940C
:1052A0008091DE059091DF05A091E005B091E105C8
:1052B00026B5A89B05C02F3F19F00196A11DB11D71
:1052C0003FBF6627782F892F9A2F620F711D811D8E
:1052D000911D42E0660F771F881F991F4A95D1F7ED
:1052E0000895CF92DF92EF92FF92CF93DF936B01FD
:1052F0007C010E944E29EB01C114D104E104F104A8
:1053000079F00E944E296C1B7D0B683E7340A0F320
:1053100081E0C81AD108E108F108C851DC4FECCF90
:10532000DF91CF91FF90EF90DF90CF900895789428
:1053300084B5826084BD84B5816084BD85B582609A
:1053400085BD85B5816085BDEEE6F0E08081816038
:105350008083E1E8F0E01082808182608083808138
:1053600081608083E0E8F0E0808181608083E1EB10
:10537000F0E0808184608083E0EBF0E080818160F8
:105380008083EAE7F0E080818460808380818260AE
:105390008083808181608083808180688083109297
:1053A000C1000895833081F028F4813099F0823073
:1053B000A1F008958630A9F08730B9F08430D1F497
:1053C000809180008F7D03C0809180008F778093D3
:1053D0008000089584B58F7702C084B58F7D84BD29
:1053E00008958091B0008F7703C08091B0008F7DC9
:1053F0008093B0000895CF93DF9390E0FC01ED50CF
:10540000F44F2491FC01E95FF34F8491882349F123
:1054100090E0880F991FFC01E15DF34FA591B491D5
:105420008B5D934FFC01C591D4919FB7611108C06A
:10543000F8948C91209582238C93888182230AC0D2
:10544000623051F4F8948C91322F309583238C93F1
:105450008881822B888304C0F8948C91822B8C9352
:105460009FBFDF91CF910895A1E0B0E0EAE3FAE2B7
:105470000C94F52E282F30E0F901E152F44F84917D
:10548000F901ED50F44F1491F901E95FF34F0491E4
:105490000023C9F0882321F069830E94D229698101
:1054A000E02FF0E0EE0FFF1FEB5DF34FA591B491FD
:1054B0009FB7F8948C91611103C01095812301C0AE
:1054C000812B8C939FBF2196E4E00C94112FCF93F6
:1054D000DF93282F30E0F901E152F44F8491F90174
:1054E000ED50F44FD491F901E95FF34FC491CC230F
:1054F00091F081110E94D229EC2FF0E0EE0FFF1FF6
:10550000E55EF34FA591B4912C912D2381E090E0BD
:1055100021F480E002C080E090E0DF91CF91089517
:105520008E3008F08E50877020919D0190E4299F65
:1055300090011124822B80937C0080917A008064FA
:1055400080937A0080917A0086FDFCCF809178006C
:105550002091790090E0922B0895A0E0B0E0E3EB79
:10556000FAE20C94F12E6C017A01EB01E60EF71EC3
:1055700000E010E0CE15DF0561F06991D601ED91F4
:10558000FC910190F081E02DC6010995080F191FCB
:10559000F1CFC801CDB7DEB7E8E00C940D2F61154F
:1055A000710589F0DB010D900020E9F7AD01415054
:1055B0005109461B570BDC01ED91FC910280F381F0
:1055C000E02D0995089580E090E00895EF92FF9214
:1055D0000F931F93CF93DF938C01FB01C0E0D0E0CA
:1055E00064917F018FEFE81AF80A662361F0D80111
:1055F000ED91FC910190F081E02DC8010995C80F53
:10560000D91FF701EDCFCE01CDB7DEB7E6E00C94A0
:105610000F2F0E94CF2A0895DC01ED91FC9101909B
:10562000F081E02D099508950F931F93CF93DF9399
:10563000EC016DE00E940C2B8C016AE0CE010E940F
:105640000C2B800F911FDF91CF911F910F91089527
:105650000F931F93CF93DF93EC010E94E62A8C01F6
:10566000CE010E94142B800F911FDF91CF911F91CB
:105670000F9108950F931F93CF93DF93EC010E9436
:10568000CF2A8C01CE010E94142B800F911FDF9135
:10569000CF911F910F9108950F931F93CF93DF9395
:1056A000EC010E940C2B8C01CE010E94142B800F68
:1056B000911FDF91CF911F910F910895A1E2B0E06A
:1056C000E4E6FBE20C94ED2E7C01C42EE52FCB0129
:1056D000D22E19A221E02D1510F02AE0D22E8E0133
:1056E0000F5D1F4F8D2C912CA12CB12C6C2D7E2F7A
:1056F000A50194010E94A62E8C2DD29E8019112402
:10570000015011098A3010F4805D01C0895CF801F4
:105710008083211531054105510521F0C22EE32F6B
:10572000CA01E4CFB801C7010E94CF2AA196ECE0DC
:105730000C94092FA0E0B0E0E0EAFBE20C94F12E1B
:10574000EC016A017B012115310541F4E881F98101
:105750000190F081E02D642F09951DC02A3031059C
:10576000A9F477FF12C06DE20E940C2B8C01442734
:105770005527BA014C195D096E097F092AE0CE014F
:105780000E945E2B800F911F06C02AE0B701A60180
:10579000CE010E945E2BCDB7DEB7E8E00C940D2F52
:1057A0009A01AB01662757FD6095762F0E949A2BD0
:1057B00008950F931F93CF93DF93EC019A01AB01F0
:1057C000662757FD6095762F0E949A2B8C01CE019B
:1057D0000E94142B800F911FDF91CF911F910F9189
:1057E00008952115310549F4DC01ED91FC910190FA
:1057F000F081E02D642F099508950E945E2B089595
:105800009A01462F50E060E070E00E94F12B08956D
:105810009A01AB0160E070E00E94F12B08950F93B4
:105820001F93CF93DF93EC010E94F12B8C01CE01EB
:105830000E94142B800F911FDF91CF911F910F9128
:1058400008950F931F93CF93DF93EC019A01AB015F
:1058500060E070E00E94F12B8C01CE010E94142BBD
:10586000800F911FDF91CF911F910F9108950F939A
:105870001F93CF93DF93EC019A01462F50E060E035
:1058800070E00E94F12B8C01CE010E94142B800F3E
:10589000911FDF91CF911F910F910895FC012485F5
:1058A0003585F901E05CFF4F80819181F901EE5B64
:1058B000FF4F20813181821B930B8F7399270895AD
:1058C000FC0184859585FC01E05CFF4F408151819E
:1058D000FC01EE5BFF4F208131814217530741F0FD
:1058E0000190F081E02DE80FF91F808190E008958C
:1058F0008FEF9FEF0895FC0184859585FC01E05CA6
:10590000FF4F40815181FC01EE5BFF4F20813181CF
:105910004217530779F0A081B181A80FB91F8C916C
:10592000208131812F5F3F4F2F73332731832083B5
:1059300090E008958FEF9FEF0895FC0181A18823E7
:1059400029F0A489B5898C9186FFFBCF11A2089517
:10595000CF93DF93FC0126853785D901A05CBF4F2B
:105960008D919C91119701968F739927E901CE5BD8
:10597000DF4F4881598184179507D9F30D90BC9169
:10598000A02DA20FB31F6C93A685B785A05CBF4F57
:1059900011969C938E93A689B7892C9181E090E013
:1059A000078C02C0880F991F0A94E2F7282B2C93CA
:1059B00081E081A30488F589E02D80818064808363
:1059C00081E090E0DF91CF91089508951F920F92AA
:1059D0000FB60F9211242F933F934F938F939F9362
:1059E000EF93FF938091C00082FD1CC04091C600E0
:1059F000809188069091890601968F73992720914E
:105A00008A0630918B068217930771F0E091880621
:105A1000F0918906E85BF94F408390938906809363
:105A2000880602C08091C600FF91EF919F918F91EF
:105A30004F913F912F910F900FBE0F901F9018958F
:105A400082EE95E00E944E2C892B11F00E94E52CED
:105A500008951F920F920FB60F9211242F933F9328
:105A60008F939F93EF93FF932091440630914506C7
:105A700080914606909147062817390731F48091A6
:105A8000C1008F7D8093C10014C0E0914606F09163
:105A90004706EC5FF94F20818091460690914706BA
:105AA00001968F739927909347068093460620931B
:105AB000C600FF91EF919F918F913F912F910F9091
:105AC0000FBE0F901F901895A0E0B0E0EAE6FDE24F
:105AD0000C94ED2EFC011382128288EE93E0A0E07C
:105AE000B0E084839583A683B7838CEB93E09183A6
:105AF00080837587648757874687318B208B138B0C
:105B0000028BF58AE48AD78AC68AB18EA08E938EDC
:105B1000828E8F85848F8889858F8989868F8A89EF
:105B2000878F8B8980A3ECE00C94092FCF92DF92B2
:105B3000EF92FF92CF93DF93EC016A017B01411555
:105B400081EE580761057105F9F0EC89FD8981E066
:105B500090E008A002C0880F991F0A94E2F78083A2
:105B600060E079E08DE390E0A70196010E94A62E07
:105B70002150310941095109569547953795279587
:105B8000211580E1380798F0EC89FD89108260E8E2
:105B900074E88EE190E0A70196010E94A62E2150A4
:105BA0003109410951095695479537952795E88957
:105BB000F9893083EA89FB89208319A2EE89FF895C
:105BC000408181E090E09C010C8C02C0220F331FC9
:105BD0000A94E2F7422B4083EE89FF8940819C01C1
:105BE0000D8C02C0220F331F0A94E2F7422B408330
:105BF000EE89FF8940819C010E8C02C0220F331F69
:105C00000A94E2F7422B4083EE89FF8920810F8CB2
:105C100002C0880F991F0A94E2F78095822380833F
:105C2000DF91CF91FF90EF90DF90CF9008958F920A
:105C30009F92AF92BF92CF92DF92EF92FF920F931B
:105C40001F9381E08F9385E08F9387E08F9383E0AC
:105C50008F9384E08F93E6EC8E2E912CF2ECAF2E96
:105C6000B12CA1ECCA2ED12CB0ECEB2EF12C04EC13
:105C700010E025EC30E044E056E068E476E082EEA7
:105C800095E00E94642D0F900F900F900F900F9051
:105C90001F910F91FF90EF90DF90CF90BF90AF904A
:105CA0009F908F9008950E9497290E94D522C0E26C
:105CB000DDE20E9489252097E1F30E94202DF9CF93
:105CC000A29FB001B39FC001A39F700D811D11243D
:105CD000911DB29F700D811D1124911D08950E9488
:105CE000602EA59F900DB49F900DA49F800D911DD7
:105CF00011240895B7FF0C946F2E0E946F2E821B03
:105D0000930B0895DB018F939F930E946F2EBF9199
:105D1000AF91A29F800D911DA39F900DB29F900DFA
:105D20001124089597FB072E16F4009407D077FDF1
:105D300009D00E94242F07FC05D03EF49095819550
:105D40009F4F0895709561957F4F0895A1E21A2E97
:105D5000AA1BBB1BFD010DC0AA1FBB1FEE1FFF1F0F
:105D6000A217B307E407F50720F0A21BB30BE40B5F
:105D7000F50B661F771F881F991F1A9469F76095A6
:105D80007095809590959B01AC01BD01CF01089560
:105D9000052E97FB1EF400940E94DF2E57FD07D0BE
:105DA0000E94A62E07FC03D04EF40C94DF2E5095D3
:105DB0004095309521953F4F4F4F5F4F08959095F7
:105DC0008095709561957F4F8F4F9F4F08952F92CB
:105DD0003F924F925F926F927F928F929F92AF927B
:105DE000BF92CF92DF92EF92FF920F931F93CF93C8
:105DF000DF93CDB7DEB7CA1BDB0B0FB6F894DEBF5F
:105E00000FBECDBF09942A88398848885F846E8484
:105E10007D848C849B84AA84B984C884DF80EE80CE
:105E2000FD800C811B81AA81B981CE0FD11D0FB6D7
:105E3000F894DEBF0FBECDBFED010895EE0FFF1F3A
:105E40000590F491E02D0994AA1BBB1B51E107C0FA
:105E5000AA1FBB1FA617B70710F0A61BB70B881FFA
:105E6000991F5A95A9F780959095BC01CD01089589
:105E70008F929F92AF92BF92CF92DF92EF92FF925A
:105E8000CF93DF93EC01688179818A819B816115D1
:105E900071058105910521F464E279ED8BE597E0C8
:105EA0002DE133EF41E050E00E94C82E49015A0134
:105EB0009B01AC01A7EAB1E40E946F2E6B017C014B
:105EC000ACEEB4EFA50194010E947D2EC60ED71E44
:105ED000E81EF91EF7FE06C081E0C81AD108E108E5
:105EE00080E8F80AC882D982EA82FB82C701B6013B
:105EF0009F77DF91CF91FF90EF90DF90CF90BF9091
:105F0000AF909F908F9008950E94382F089586E05B
:105F100091E00E94382F0895609306017093070165
:105F2000809308019093090108952F923F925F9208
:105F30006F927F928F929F92AF92BF92CF92DF9299
:105F4000EF92FF920F931F93CF93DF938B01EA01A0
:105F50006115710521F0DB018C9311969C932097BC
:105F600039F09E01225031092332310508F0D8C0A2
:105F70007C016701BFEFCB1ADB0A5601F701608095
:105F8000862D90E00E94C730892B11F07601F1CF69
:105F9000FDE26F120AC0570182E0A80EB11CD701C2
:105FA00011966C90772473940BC0BBE26B1207C000
:105FB0005701E2E0AE0EB11CD70111966C90712C26
:105FC000CE018F7E892B89F4B0E36B1237C0F501C7
:105FD00080818F7D8835D1F46180F2E0AF0EB11CF5
:105FE000872D8260782EC0E1D0E0CA30D10551F112
:105FF000C031D10521F0C830D10599F409C0CC24B5
:10600000CA94DC2CEC2CAFE0FA2E22C0209769F762
:10601000C8E0D0E0CC24CA94DC2CEC2CFFE1FF2EAD
:1060200017C06FEF7FEFCB019E01442737FD4095EE
:10603000542F0E94A62E69017A010AC02097A9F662
:10604000CAE0D0E0E9E9CE2EDC2CEC2CE9E1FE2E12
:10605000F50160E020E030E0A9014E01AA2497FCA0
:10606000A094BA2C1F0170ED572E560CA9E0A5156F
:1060700070F48FEB860D8A3118F499EC592E06C016
:106080008FE9860D8A3148F589EA582E560C852D00
:1060900090E08C179D070CF56F3FD9F0C216D30620
:1060A000E406F50698F0C501B4010E94822E9B011A
:1060B000AC01852D90E0A0E0B0E0280F391F4A1F09
:1060C0005B1F281739074A075B0710F46FEF01C001
:1060D00061E03196D1016C90C5CF0115110551F0E9
:1060E000662311F0319703C071FE04C03297D801C6
:1060F000ED93FC9370FE07C0509540953095219527
:106100003F4F4F4F5F4F67FF10C082E290E0909388
:106110008D0680938C066FEF7FEF8FEF9FEF07C0A8
:1061200060E070E080E090E002C0B901CA01DF9158
:10613000CF911F910F91FF90EF90DF90CF90BF9084
:10614000AF909F908F907F906F905F903F902F9037
:106150000895FC0188279927E89421912032E9F3DA
:10616000293010F02E30C8F32B3241F02D3239F4A3
:10617000689404C00E94FB30820F911D219120532E
:106180002A30C0F31EF4909581959F4F0895911188
:1061900050C0803219F089508550D0F7089548ECEE
:1061A00053E00E94D4300895FA01A191B081009784
:1061B00019F41097E1F0CD01DC01CD010D90002024
:1061C00011F4C00113C0FB012191222319F0201505
:1061D000D9F7F3CFFB012191201519F41E921196E6
:1061E00006C02223C1F70D900020A1F7D001FA01CB
:1061F000A193B08308957AE0979F902D879F802D7B
:10620000910D11240895F999FECF92BD81BDF89AA0
:10621000992780B50895262FF999FECF1FBA92BD10
:1062200081BD20BD0FB6F894FA9AF99A0FBE019677
:0C6230000895992788270895F894FFCF5F
:10623C0000008E06200001000000FF00020002009A
:10624C000200020002000200020002000200020032
:10625C00020002000200020002000280250000057C
:10626C00400AA1204EA50020244EA52C2330C0129C
:10627C0000001A400AA1204EA5001B1E27522C23F9
:10628C00308025000005400AA1204EA50020244E98
:10629C00A52C2330004B000006400AD0009D49007D
:1062AC007B289D492C233000E1000005400A450164
:1062BC00D7DC03B81E0EBF00232E48E801008A402D
:1062CC000A6001555502AD1E20000023C801545828
:1062DC002074696D656F75742100596573004E6F7C
:1062EC00002C00386368004E2F41002C205B005DB1
:1062FC002028002900486F70206368616E6E656C01
:10630C00200020402000456E746572696E67206124
:10631C0064617074697665206368616E6E656C206B
:10632C0073656C656374696F6E2C207069636B693F
:10633C006E673A007363616E6E6572206D6F646593
:10634C00004E4F5420454E41424C45440053656E1F
:10635C0064696E672073657474696E677320746FFB
:10636C002052580A00526573657474696E67207305
:10637C00657474696E6773206F6E2052580A004101
:10638C00626F727465642065646974730A00696E67
:10639C0076616C69642073656C656374696F6E00FB
:1063AC000D0A496E76616C696420696E7075742093
:1063BC002D20646973636172646564210700536501
:1063CC007474696E677320736176656420746F20D2
:1063DC00454550524F4D0A0052657665727465649E
:1063EC002073657474696E67732066726F6D2045D7
:1063FC004550524F4D0A004C6F61646564206661D4
:10640C0063746F72792064656661756C74730A00CD
:10641C004B657920616E64206368616E6E656C7388
:10642C002072616E646F6D697A65640A004F7065E5
:10643C006E4C52536E672054582073746172746999
:10644C006E672000206F6E20485720006D6F6475BA
:10645C006C65206C6F636B65643F00342B340038C3
:10646C0000382B340031320031322B3400313600FD
:10647C0050504D0052535349005344410053434C28
:10648C0000525844005458440041494E004C424577
:10649C0045500053504B54524D00534255530053EA
:1064AC00554D44004C4C494E440000070B0C101148
:1064BC001500B7012B032F033103350338033D03BC
:1064CC00B7014003440349034D03510355035903DA
:1064DC005D0363036A036F0374038D028D028D02E7
:1064EC008D02160A1322312900000000A82CAD2AB7
:0864FC004E2C7B2C602C9D2C22
:00000001FF
